:020000040000FA
:020000005B287B
:08000800F000030E8312F10069
:1000100016218B180D280B181628061C48282214A8
:10002000861F0430861B0830A500512823080606C9
:1000300003194828A300231A2428A31A2B28231BBA
:100040003228A31B39284828061E4828221C0530C0
:10005000221848284628861E4828221C06302218C6
:1000600048284628061B4828221C4828221005300C
:100070004628861B3C284128221C013022180330C8
:100080004628221C0730221804304628A500512893
:100090000608A3008B100B10710E8300F00E700E7B
:1000A00009000608A3008B100B10710E8300F00EE0
:1000B000700E8B1780281F149F141F158316FD3098
:1000C00085008312850183163F3092008312003031
:1000D0009500970197151715831686118312121034
:1000E000921012150608A300A5012210831601170D
:1000F00083120B168B158B100B108B170E210E21F4
:10010000013025020319A528033025020319AC2864
:10011000023025020319B328043025020319BA2836
:10012000073025020319EC28053025020319A528FC
:10013000063025020319B3280830250203190529C2
:1001400085141621851016218028403015020319C8
:10015000C128950A1A21A528403015020319C12883
:10016000950A1E21AC28003015020319C1289503F9
:100170001A21B328003015020319C12895031E2146
:10018000BA28053025020319EC2806302502031988
:10019000CB28A50180280E210E210E21D320D320AB
:1001A000D320A501802895014030950085141621A3
:1001B000162195018510162104309507162120304F
:1001C0001502031DDC288514162104309502162122
:1001D000031DE5288510080095080319C128403043
:1001E00015020319F628950A1A21EF2885100D30FB
:1001F000A4000E210E210E210E218514162185103A
:10020000A40BF9280230A500802814301502031928
:100210000C2995031E210529A5018028FA30A0008C
:10022000222108006430A000222108003230A00002
:10023000222108002830A000222108000A30A00056
:1002400022210800F930A100000000000000000099
:10025000000000000000000000000000000000009E
:1002600000000000000000000000A10B2429A00BEA
:040270002229080037
:02400E00023F6F
:104200004B0046005A002D0049006E006E0065000C
:104210006E006C006900630068007400640069004F
:104220006D006D00650072002000760033002000F4
:1042300028006300290032003000300034002000E4
:1042400062007900200063006F006F006C00630063
:104250006800690070002E006400650020002000E6
:00000001FF
